:1000000001308A00DC290000D3346D38EC32202A1C
:10001000E832F236EF36653AE8327210A0060A008E
:10002000532A412BA0126C2CA0060A00C432EC32D9
:10003000EE372019351B3A10253658102838F2377C
:10004000E3326E3AE1140D050001D337F531653A1C
:10005000A016A039EF3AE332F417B21A361DA012F7
:100060006C2CA0060A00CC29421DA0126C2C0D0598
:10007000000083168611831286110830F80040288C
:100080000000F8175128F813AD0C03188615031C4F
:100090008611781751287813F80B44284F28000050
:1000A00086153F308400840B53280000F81B43283A
:1000B000781B4B280800831603178C170C140000BC
:1000C000000083120C087F3903199F280313A9002D
:1000D00003170D080313AA0003170F080313AB003F
:1000E0002908AD0039202A0803178D0003132B08B7
:1000F00003178F0083168C170C1400000000831266
:100100000C0D0E0D7F3903199F280313A900031747
:100110000D080313AA0003170F080313AB002908E7
:10012000AD0039202A0803178D0003132B0803178D
:100130008F008D0A03198F0A03135B28031703131B
:100140008A110A12442A0830F8000000861083162B
:10015000861000008312A90D0610031CB228831616
:10016000061483120318B728831606108312831609
:1001700086148312861CBA28F80BA5280000861066
:1001800083168610000006140000000086148312F7
:10019000861CC828F80100000618781486108316FB
:1001A0008610831206108316061083120800293069
:1001B0008400831300080319EA280230F800F701CD
:1001C000F70BE028F80BDF289730F700F70BE6284D
:1001D000800BDD2808002C08F8012B020318F328F7
:1001E0002B08F700FF28F7010830AD00AB0DF70D25
:1001F0002C0877020318F700F80DAD0BF62808005D
:1002000078082908AB006430AC00EB207708A9001F
:1002100078083030031D1329AA1C1A29AA191A2993
:100220002A1A20301629AA112A122A14F807780847
:10023000AD0039202908AB000A30AC00EB2077086C
:10024000A90078083030031D2B29AA192F292A1C50
:100250002F292A1A2030F8077808AD0039203030CD
:10026000A9072908AD0039208A110A12072B083086
:10027000AA007708AB0083160614000086148312C8
:10028000861C402906180314061C0310F80D0000F4
:100290008316861083128610AA0B3B298316061438
:1002A0000000831206102B08031959298316061023
:1002B00083120000831686148312861C5D290000B9
:1002C000861083168610000083120610831606100F
:1002D00083128A110A12442B831603178C170C14ED
:1002E0000000000003189B2983120C087F390313B8
:1002F000AA0003170D080313AB0003170F0803131D
:10030000AC002A08AD0039202B0803178D00031319
:100310002C0803178F0083168C170C1400000000A4
:1003200083120313A90B95299829831603179B2978
:10033000BA298316031783120C0D0E0D7F39031390
:10034000AA0003170D080313AB0003170F080313CC
:10035000AC002A08AD0039202B0803178D000313C9
:100360002C0803178F008D0A03198F0A031003133B
:10037000A90B6C290800AA1BCD290F30F700290E04
:10038000F7050A3077020318C8293030F707CA2961
:100390002A08F7077708AD0039200F30A9050A3081
:1003A00029020318D5293030D729AA132A08A9070A
:1003B0002908AD0039200800840183131F3083050C
:1003C000713083168F000F088611831286158316ED
:1003D00003170908C039890003131F129F12003048
:1003E000031788008312870188018901FF300313F6
:1003F000A000831603170908C039890003131F12D0
:100400009F12003003178800831203131F139F13DA
:1004100083169F1383121F149412A01220088316B0
:100420008700831220162008831687008312A011EC
:100430002008831687000130831294000030831651
:1004400094000108C73908388100831290010030F8
:10045000F8009200003083169200831220152008C5
:10046000831687008312970183169B019C0101303C
:100470009D008312031787018801890104308D00D4
:1004800000308F0003135B288316061400008614C7
:1004900000008312061083160610000083128610D7
:1004A00083168610AA308312A900A3206130A90008
:1004B000A320831606140000861400008312861CF5
:1004C0005F2A06108316061000008312861083161A
:1004D0008610AA308312A900A320A901A3208316A5
:1004E0000610000086148312861C742A0000782AE5
:1004F000000083160614000001308312A900D720E3
:10050000831606140000861400008312061083165A
:10051000061000008312861083168610AA308312FC
:10052000A900A3203E30A900A320831606140000D2
:10053000861400008312861C9B2A06108316061060
:1005400000008312861083168610AA308312A90039
:10055000A3204030A900A3208316061000008614B3
:100560008312861CB12A0000B52A000083160614E7
:10057000000001308312A900D72083160614000062
:1005800086140000831206108316061000008312E2
:10059000861083168610AA308312A900A3203F304C
:1005A000A900A320831606140000861400008312FD
:1005B000861CD82A061083160610000083128610A7
:1005C00083168610AA308312A900A320A901A320B4
:1005D00083160610000086148312861CED2A000084
:1005E000F12A000083160614000001308312A900CE
:1005F000D7204030A800A401A301A8002808603C2F
:10060000031C722B2808A9001B30AA0000290D30FA
:10061000AD0039200A30AD003920831606100000E5
:1006200086148312861C122B0000162B00008316E2
:100630000614000006140000861400008312061041
:100640008316061000008312861083168610AA30C7
:100650008312A900A3202808A900A320831606144A
:100660000000861400008312861C342B06108316AB
:10067000061000008312861083168610AB3083129A
:10068000A900A320F70137297808A10083160610D6
:10069000000086148312861C4B2B00004F2B000099
:1006A0008316061400001030831203178D000030EB
:1006B0008F00031005300313A9006C212108A90045
:1006C0003730AA00BB212030AD0039200D30AD00FD
:1006D00039200A30AD0039202108A3070318A40AE5
:1006E000A80AFE2A2408A6002308A5002608A500BB
:1006F000A601163003178D0000308F0003100C3058
:100700000313A9006C212608A9003730AA00BB21D9
:100710002508A9003730AA00BB211D3003178D0022
:1007200000308F0003140D300313A9006C2125083D
:100730002302A5002608031C260FA02B2408A12BAA
:100740002402A600253003178D0000308F0003100F
:1007500015300313A9006C212608A9003730AA0020
:10076000BB212508A9003730AA00BB212030AD00ED
:1007700039200D30AD0039200A30AD003920250870
:10078000A700333003178D0000308F0003100530B1
:100790000313A9006C212708A9003730AA00BB2148
:1007A0000D30AD0039200A30AD0039206430A90089
:0407B000D7206300EB
:04400E00F52CFF3F4F
:00000001FF
